:100000005F2AFF3FFF3FFF3F8D000F088C000B1161
:1000100002308506203081008D008F0E0C0E0830D6
:100020008E00851C1128051D112803108D0C031846
:100030003928851105191A288514051D1D288E0BD0
:1000400011284128133084000F088D0008308E00DD
:100050000D088F0064008D3062000310800D031CBA
:10006000332856223428A0208E0B2828840A900B8F
:100070002628051085183A280515851C3D288E0B65
:100080001128851C4128051D412809003F340634EC
:100090005B344F3466346D347D3407347F346F34D1
:1000A00002300D0203197F2A03300D0203197D2A45
:1000B00004300D0203197F2A05300D020319932A1B
:1000C00006300D0203197F2A07300D0203197F2A1B
:1000D00008300D020319AB2A09300D0203197F2ADB
:1000E0000A300D020319D12A0B300D0203197F2AA1
:1000F0008207000000000000000000000000000077
:1001000000000000000000000000000000000000EF
:10011000000000000000000000000000080086143D
:10012000912892289328942895289628000000006A
:1001300099289A289B289C289D288F0B8F28080097
:100140008614110878200000120878208F0BA02850
:10015000080086140512851DC928851C861085187F
:1001600086148D0C8D0BB1288D0164008D306200DA
:1001700008308E008518C728051DBA288511031080
:100180008D0C851CC12885158E0BBA280800051911
:10019000BA28051003148D0C051DCC2805148E0BF0
:1001A000BA280800283463342934203453346134A5
:1001B0006D34693420344B346834613477346134BD
:1001C0006D34203473344B346834613477346134A3
:1001D0006D34403462346934673466346F346F345C
:1001E00074342E3463346F346D340E308F008610C7
:1001F0000B30782086140F3078208F0BF7280800FA
:10020000493452342D344C3469346E346B342034D8
:10021000763465347234733469346F346E34203418
:1002200032342E343034003464008D3062000830B3
:100230008E00851C1929051D192903108D0C031822
:100240002A290510051922290514051D25298E0BBB
:1002500019293229851185182B298515851C2E29E8
:100260008E0B1929851C3229051D322908000C34F2
:10027000843485347B342B344C341A34BD344134CB
:100280005734363420342C3458349C3420349B304A
:100290008C0064008D30620000008C0B4C2908003B
:1002A0000E308F0086140B30782000000F3078203D
:1002B0008F0B522908000E341134113411341134CB
:1002C00011340E3404340C3404340434043404344F
:1002D0000E340E34113401340234043408341F3423
:1002E0000E34113401340634013411340E34023426
:1002F00006340A3412341F34023402341F341034EA
:100300001E340134013411340E340E3411341034DF
:100310000E34113411340E341F34013401340234DC
:100320000234043404340E34113411340E341134D4
:1003300011340E340E34113411340F3401341134AD
:100340000E340034003408340434023400340034F1
:1003500002340434083400340034003400340034EF
:10036000003400340E34113411341F34113411347C
:1003700011341F3411341134113411341134113447
:100380000E341E34113411341134113411341E342E
:10039000113411341E34113411341E34103410341D
:1003A00010341034103410341F34103410341C3412
:1003B000103410341F34103410341C341034103402
:1003C00010340134013401340134013411340E3459
:1003D000113410341334113411340E3411341134F7
:1003E0001134153413340E34113410340E340134F6
:1003F00011340E34113410341034103411340E34DE
:10040000043404340434043404340E341134123407
:10041000143418341434123411341B341534113498
:100420001134113411341934153413341134113496
:1004300011340A340434043404341E3411341134B5
:100440001E34113411341134113411340A3404348B
:100450000A34113411341134113415341B3411346D
:100460001F34013402340434083410341F3404348B
:100470000434043404340434043407308F00522923
:1004800004308F0052297E3430346D347934333463
:100490005B345F3470347F34733477341F344E34BC
:1004A0003D344F3447340C308F00522986101108E8
:1004B00078208614120878208F0B562A08001630F0
:1004C0006500803066008D306200850186018614EB
:1004D000851505148B1300309300003094006400E0
:1004E0008D3062000610051E7D2A051D7A2A851CA6
:1004F000932A6F2A8518932A6F2A861B6F2A8D01EB
:1005000008308E003D220614051A6F2A5021051E60
:100510000310051A03148D0C8E0B862A5021051A20
:100520006F2A1421752A0614861BAB2AB4200830C2
:100530008E00F52003108D0C0318A22AF5208E0BD7
:100540009A2AA52A50218E0B9A2AF5205322472158
:10055000472147216F2AB4200D0890008C00B42059
:100560000D088F00B4200D089100B4200D089200F2
:1005700013308400B4200D088000840A8C0BBA2A42
:10058000133084000F088D0008308E000D088F0096
:1005900064008D3062000310800D031CD12A5622A6
:1005A000D22AA0208E0BC62A840A900BC42A472187
:1005B0006F2A20348834433412346534543443343D
:1005C0002134983402340434B834A434C0340634AA
:1005D000243488342634FF3FFF3FFF3FFF3FFF3F77
:1005E000FF3FFF3FFF3FFF3FFF3FFF3FFF3FFF3F1B
:1005F000FF3FFF3FFF3FFF3FFF3FFF3FFF3FFF3F0B
:10060000FF3FFF3FFF3FFF3FFF3FFF3FFF3FFF3FFA
:10061000FF3FFF3FFF3FFF3FFF3FFF3FFF3FFF3FEA
:02400E00FD3F74
:1042000000000000000000000000000000000000AE
:10421000000000000000000000000000000000009E
:10422000000000000000000000000000000000008E
:10423000000000000000000000000000000000007E
:10424000000000000000000000000000000000006E
:10425000000000000000000000000000000000005E
:10426000000000000000000000000000000000004E
:10427000000000000000000000000000000000003E
:00000001FF
